:020000040000FA
:0400000083016728E9
:08000800FF00030E8301A000BC
:100010000A08A1000408A2008A010313831222081F
:10002000AC002308AD002408AE002508AF00260868
:10003000B0002708B1002808B2002908B3002A0838
:10004000B4002B08B5008B18F72B2C08A2002D0844
:10005000A3002E08A4002F08A5003008A600310830
:10006000A7003208A8003308A9003408AA00350800
:10007000AB002208840021088A00200E8300FF0EB6
:100080007F0E0900031383122408270203184D284A
:1000900003194D280130A7000034A70100340313D1
:1000A000831224082702031C5A2803195A280130F6
:1000B000A7000034A7010034031383122408270289
:1000C000031D65280130A7000034A7010034031385
:1000D00083128316DA3081006400DA3081008312E3
:1000E000103083168500073086000A308312CF0057
:1000F000C301C401C501C601C701C801C901CA01C4
:10010000CB01B601B701B801BB01BC01B9010510B3
:10011000851005118613061386120612861101300A
:10012000BA008B170B1701170B160313831239082C
:10013000A9000130A7002908A4005C200313831242
:100140000130A7062708271CA62895280313831229
:100150006400031383120618C90A0319EF2B8618CB
:10016000CA0A0319EF2B0619CB0A0319EF2B00005B
:10017000000000003918A9283A08A9000130A7009A
:100180002908A4005C20031383122708271C452993
:100190004908A9009630AA004F082A02A70029089A
:1001A000A4004220031383122708A9004908AA00CB
:1001B0009630AB004F082B07A7002A08A4004F2059
:1001C0000313831227082908A705271CEA284908D2
:1001D000CC00EE28031383129630CC000313831255
:1001E0004A08A9009630AA004F082A02A700290849
:1001F000A4004220031383122708A9004A08AA007A
:100200009630AB004F082B07A7002A08A4004F2008
:100210000313831227082908A705271C12294A0857
:10022000CD001629031383129630CD0003138312D9
:100230004B08A9009630AA004F082A02A7002908F7
:10024000A4004220031383122708A9004B08AA0028
:100250009630AB004F082B07A7002A08A4004F20B8
:100260000313831227082908A705271C3A294B08DE
:10027000CE003E29031383129630CE00031383125F
:10028000BA01C901CA01CB019528031383128B134C
:100290000B13BD01BE01BF01C001C101C2014D0868
:1002A000A9003C302907A9004A08A7002908A40092
:1002B0004220031383122708A9004A08AA004D0808
:1002C000AB004F082B07A7002A08A4004220031305
:1002D000831227082908A705271C70290130BE00B2
:1002E000031383124D08A9004F082907A9004A08E3
:1002F000A7002908A4004F20031383120130A7068A
:100300002708A9004A08AA004D08AB004F082B0295
:10031000A7002A08A4004F20031383120130A70668
:1003200027082908A705271C97290130C1000313B6
:1003300083124D08A9003C302902A9004A08A700F1
:100340002908A4004F20031383122708A9004A0894
:10035000AA004D08AB004F082B02A7002A08A400F2
:100360004F200313831227082908A705271CBA2941
:100370000130BD00031383124C08A9003C3029074B
:10038000A9004908A7002908A400422003138312EA
:100390002708A9004908AA004C08AB004F082B0702
:1003A000A7002A08A4004220031383122708290863
:1003B000A705271CDD290130BF00031383124C0859
:1003C000A9004F082907A9004908A7002908A40087
:1003D0004F20031383120130A7062708A9004908FC
:1003E000AA004C08AB004F082B02A7002A08A40063
:1003F0004F20031383120130A70627082908A705F9
:10040000271C042A0130C200031383124C08A900E0
:100410003C302902A9004908A7002908A4004F2060
:10042000031383122708A9004908AA004C08AB004F
:100430004F082B02A7002A08A4004F2003138312A1
:1004400027082908A705271C272A0130C000031305
:1004500083124E08A9003C302907A9004B08A700C9
:100460002908A4004220031383122708A9004B087F
:10047000AA004E08AB004F082B07A7002A08A400CB
:1004800042200313831227082908A705271C492A9D
:100490000514031383124E08A9004F082907A90069
:1004A0004B08A7002908A400422003138312270841
:1004B000A9004B08AA004E08AB004F082B02A7006A
:1004C0002A08A40042200313831227082908A7053D
:1004D000271C6C2A05108510031383124E08A900EF
:1004E0003C302902A9004B08A7002908A4004F208E
:1004F000031383122708A9004B08AA004E08AB007B
:100500004F082B02A7002A08A4004F2003138312D0
:1005100027082908A705271C8E2A85140313831290
:100520004B08A9005030A7002908A4004F2003134E
:1005300083122708A9004B08AA00DC30A7002A086C
:10054000A40042200313831227082908A704271CAC
:10055000AB2A05108510031383124908A9005030F7
:10056000A7002908A4004F20031383122708A9001D
:100570004A08AA005030A7002A08A4004F200313FD
:10058000831227082908A704271CCA2AEF2303136C
:100590008312E32B031383124208A9000130A70042
:1005A0002908A4005C20031383122708A90041082E
:1005B000AA000130A7002A08A4005C2003138312BC
:1005C00027082908A705271CE92A86110612861282
:1005D0000613031383123D08A9000130A700290860
:1005E000A4005C20031383122708A9004208AA0074
:1005F0000130A7002A08A4005C20031383122708F7
:100600002908A705271C082B06120613861686152F
:10061000031383123E08A9000130A7002908A40093
:100620005C20031383122708A9004208AA000130A6
:10063000A7002A08A4005C200313831227082908B6
:10064000A705271C272B86118612061606170313EB
:1006500083123F08A9000130A7002908A4005C20EC
:10066000031383122708A9004108AA000130A7003C
:100670002A08A4005C200313831227082908A70571
:10068000271C462B061286128615061703138312A3
:100690004008A9000130A7002908A4005C2003132A
:1006A00083122708A9004108AA000130A7002A08E0
:1006B000A4005C200313831227082908A705271C20
:1006C000652B86110613061686160313831240083F
:1006D000A9000130A7002908A4005C20031383129D
:1006E0002708A9003D08AA000130A7002A08A40095
:1006F0005C200313831227082908A705271C842BD5
:100700008611061206138616031383123D08A900EC
:100710000130A7002908A4005C20031383122708D6
:10072000A9003F08AA000130A7002A08A4005C2005
:100730000313831227082908A705271CA32B0612D9
:10074000861206138615031383124008A900013090
:10075000A7002908A4005C20031383122708A9001E
:100760003E08AA000130A7002A08A4005C20031359
:10077000831227082908A705271CC22B86110612F9
:1007800086120617031383123F08A9000130A70041
:100790002908A4005C20031383122708A9003E083F
:1007A000AA000130A7002A08A4005C2003138312CA
:1007B00027082908A705271CE12B86118612061396
:1007C00006160313831203138312B901C901CA0168
:1007D000CB01B601B701B8018B170B17952803138E
:1007E0008312861106128612061308000F2C0313BB
:1007F00083123908A9000030A7002908A4005C2052
:10080000031383122708271C082C0130B9000B2C76
:1008100003138312B901031383128B1025280313CA
:02082000831241
:02400E002E3F43
:00000001FF
